:0200000480007A
:100000006F008004732F2034930F80006308FF0378
:10001000930F90006304FF03930FB0006300FF038E
:10002000130F000063040F0067000F00732F2034CC
:1000300063540F006F00400093E19153171F0000BD
:1000400023223FFC6FF09FFF93000000130100008C
:10005000930100001302000093020000130300004C
:100060009303000013040000930400001305000034
:10007000930500001306000093060000130700001C
:100080009307000013080000930800001309000004
:1000900093090000130A0000930A0000130B0000EC
:1000A000930B0000130C0000930C0000130D0000D4
:1000B000930D0000130E0000930E0000130F0000BC
:1000C000930F0000732540F16310050097020000B4
:1000D000938202017390523073500018970200000F
:1000E0009382020273905230B70200809382F2FF33
:1000F0007390023B9302F0017390023A73504030C8
:100100009702000093824201739052307350203066
:100110007350303093010000970200009382C2EECA
:1001200073905230130510001315F501634C050050
:100130000F00F00F930110009308D0051305000085
:100140007300000093020000638A02007390521053
:10015000B7B2000093829210739022307350003037
:10016000970200009382420173901234732540F18C
:1001700073002030B710FF00938000F013C7F0F039
:10018000B7F300FF9383F300930120006316771CFD
:10019000B710F00F938000FF13C7000FB713F00FD5
:1001A000938303F0930130006318771AB710FF00B0
:1001B0009380F08F13C7F070B713FF00938303FF92
:1001C00093014000631A7718B7F00FF09380F000A6
:1001D00013C7000FB7F30FF09383F30F9301500091
:1001E000631C7716B7F000FF9380007093C0F07027
:1001F000B7F300FF9383F30093016000639E7014D4
:1002000013020000B710F00F938000FF13C7000F18
:10021000130307001302120093022000E31452FE9E
:10022000B713F00F938303F09301700063167312FA
:1002300013020000B710FF009380F08F13C7F07017
:1002400013000000130307001302120093022000A2
:10025000E31252FEB713FF00938303FF9301800064
:10026000631C730E13020000B7F00FF09380F000D0
:1002700013C7000F13000000130000001303070052
:100280001302120093022000E31052FEB7F30FF0A6
:100290009383F30F930190006310730C130200001B
:1002A000B710F00F938000FF13C7000F1302120066
:1002B00093022000E31652FEB713F00F938303F06E
:1002C0009301A000631A770813020000B710FF0023
:1002D0009380F0FF1300000013C7F0001302120018
:1002E00093022000E31452FEB713FF00938303FF31
:1002F0009301B0006312770613020000B7F00FF00D
:100300009380F000130000001300000013C7000FDB
:100310001302120093022000E31252FEB7F30FF013
:100320009383F30F9301C000631877029340000F8B
:100330009303000F9301D00063907002B700FF0099
:100340009380F00F13C0F070930300009301E0005E
:1003500063147000631030020F00F00F638001001F
:100360009391110093E111009308D00513850100CA
:10037000730000000F00F00F930110009308D005E8
:100380001305000073000000731000C0000000009F
:10039000000000000000000000000000000000005D
:1003A000000000000000000000000000000000004D
:0C03B00000000000000000000000000041
:1010000000000000000000000000000000000000E0
:1010100000000000000000000000000000000000D0
:1010200000000000000000000000000000000000C0
:1010300000000000000000000000000000000000B0
:081040000000000000000000A8
:040000058000000077
:00000001FF
